:100000002828A301A200FF30A207031CA307031C9A
:1000100023280330A100DF300F200328A101E83E90
:10002000A000A109FC30031C1828A00703181528FC
:10003000A0070000A10F152820181E28A01C2228A8
:100040000000222808008313831203130000080015
:1000500007309F0083168501860180308312860059
:10006000A4010730240203183C280310860C4630F4
:100070000120A40A031D3128A4010730240203181B
:1000800048280310860D46300120A40A031D3D2890
:060090003028630049283E
:02400E00503F21
:00000001FF
